:020000020000FC
:100000000DC0189518951895189518951895189568
:1000100091C01895189518951895B0C000E00EBFBE
:100020000FED0DBF00E808B901E007B907EC06B90C
:1000300002E001B903E00EBD0DEF0DBD0FE80CBDF0
:1000400001E00CB94FEE00EF0ABB0BBB07E007BBAA
:10005000DD27C4E000E3402E502E602E702E7894F1
:10006000EE24FF2420E4339A2FD097FF03C09F771C
:10007000369AFACF2223C1F73398F694E794F69490
:10008000E794F694E79404E713E12ED016940794CE
:100090001694079416940794F12CE02C32D0A4E027
:1000A000BB27022D0F70002319F40FEF0D9301C031
:1000B00011D0012D029590640DD09F7B012D0AD0A7
:1000C000002D029507D0CCCF00E205BF8895002710
:1000D00005BF0895E8E8F1E00F70E00FFB1F049101
:1000E00096FD0F7D0D930895222420E11695079526
:1000F00010F41E0C2F1C2794179407942A95B1F71F
:10010000089520E1222411240024FF27EE0CFF1C77
:10011000001C111C221C2A9509F40895E3E00291A9
:100120000D5F03FD00830081005D07FD0083E0306B
:10013000B1F7ECCF0F930FB70F930DEF0DBD0FE895
:100140000CBD0BB3006F0BBBC298099138E0C0988F
:10015000000F10F4C19A01C0C198C09A3A95B9F73E
:10016000C29A0BB3006F04230BBB440F10F04FEE89
:10017000C4E090680F910FBF0F91189504B1E00E85
:1001800005B1F01E2A95189530F32AA2E1A424F2B5
:0201900020A0AD
:00000001FF
